:020000040000FA
:1000000025000504C10C0200F00C0600000C2900BC
:10001000E7060C0A130A080A050CC90103061A0AA6
:10002000050CE9011A0A050C890043061A0A050C99
:10003000A9001A0A46050902280000000000000075
:10004000000000000000E8021D0A4604FF0C280022
:10005000290A2A0A2B0A2C0A2D0A2E0A2F0A300AEC
:10006000310A320A330A340A350A360A370A380A9C
:10007000390A3A0A3B0A3C0A3D0A3E0A3F0A400A4C
:10008000410A420A430A440A450A460A470A480AFC
:06009000E802280A080A3C
:021FFE00EB0FE7
:00000001FF
